:0200000270008C
:10800000807F0020398507006185070063850700B0
:108010006585070067850700698507000000000087
:108020000000000000000000000000006B85070059
:108030006D850700000000006F850700718507004F
:108040007385070073850700738507007385070034
:108050007385070073850700738507007385070024
:108060007385070073850700738507007385070014
:108070007385070099A007007385070073850700C3
:1080800073850700819207007385070073850700D9
:1080900041930700738507002DB007007385070023
:1080A00073850700738507007385070073850700D4
:1080B00073850700738507000000000000000000C2
:1080C00073850700738507007385070073850700B4
:1080D00073850700738507007385070000000000A3
:1080E0000000000000000000000000000000000090
:1080F0000000000000000000000000000000000080
:10810000000000000000000000000000000000006F
:10811000000000000000000000000000000000005F
:1084000010B5054C237833B9044B13B10448AFF3CE
:1084100000800123237010BD882C00200000000084
:1084200024D9070008B5034B1BB103490348AFF338
:10843000008008BD000000008C2C002024D907001B
:10844000154B002B08BF134B9D46A3F5803A002126
:108450008B460F461348144A121A00F063F80F4B6C
:10846000002B00D098470E4B002B00D098470020DF
:10847000002104000D000D48002802D00C48AFF385
:10848000008000F02BF82000290000F071FD00F0C2
:1084900011F800BF00000800807F002000000000ED
:1084A00000000000882C0020B838002000000000E8
:1084B0000000000008B5074B044613B10021AFF3DC
:1084C0000080054B1868836A03B19847204600F086
:1084D00031F800BF0000000084D4070070B50D4DD6
:1084E0000D4C641BA4100026A64209D10B4D0C4C68
:1084F00004F0BCFF641BA4100026A64205D170BD89
:1085000055F8043B98470136EEE755F8043B984789
:108510000136F2E7682C0020682C0020682C00202F
:108520006C2C002002440346934200D1704703F8AC
:10853000011BF9E7FEE700BF0649074A074B9B1AF4
:1085400003DD043BC858D050FBDC02F08BFBFFF787
:1085500077FF000030D90700002C0020882C002075
:10856000FEE7FEE7FEE7FEE7FEE7FEE7FEE7FEE7E3
:10857000FEE7FEE7024A1368013B1360704700BF45
:10858000E430002030B50D490D4C8A6B85B06D4646
:1085900028465C3103F0F4FA95E80F0084E80F00F8
:1085A000084BE360084B09490022C3E9002220463A
:1085B000074A03F082FD05B030BD00BF0036002041
:1085C00058320020FD850700CC2C002058D507002C
:1085D000EC30002008B502F0D9FFBFF34F8F0549FA
:1085E000054BCA6802F4E0621343CB60BFF34F8FC0
:1085F00000BFFDE700ED00E00400FA055B689A6843
:10860000054B9A4206D1D0E9012304490132013BCE
:108610000A604B60704700BFDCD40700CC2C002000
:1086200070B5012002F0DCFD0546B8B9114B124CC3
:108630001860A36B26468BB1FFF7A4FF70B1236AC5
:1086400073B9A36963B10D4A13600C4B0C4A1868E7
:10865000002103F0D5F80B4B01221A70284670BD9B
:10866000F36A002BFAD1B369002BF7D0034B726A7F
:108670001A60EAE7E430002000360020DC300020F9
:10868000E0300020E83000202DE9F74F0B78012B77
:108690000D46164601D0062B04D12A79012A0AD1AB
:1086A0009C490A709B4A1278012A08D0022A00F0DD
:1086B0002581052422E0022AF2D007241EE0013B96
:1086C000052B00F24083DFE813F00600230043008F
:1086D0001D003E031001AB6823B3B3F5807F00F2A9
:1086E000E08000248C4B8D481C7020222146FFF72F
:1086F00019FF8B4B1C63AA689A630124204603B0C0
:10870000BDE8F08F864BDA6B72601B6CB360F4E7E8
:10871000834CAA68E06BA36B1118994204D970606E
:10872000236CB3600324E9E75C306968204404F0FB
:108730008EFEAA68E36B1344E36304F14002D5E9BB
:10874000010101F0B1F8E36B20647360236CDDE795
:10875000734ED6E90E21914240F011816E4D2B7877
:10876000002BCAD1FFF70EFF0128A2D16D4B93F861
:1087700074201C46002A00F0B38093F87A30002B56
:1087800097D06948D0E90012A9B1A2B194F8DB30C2
:1087900013B194F8DC3073B994F884305BB1D4F839
:1087A0008830342B07D194F88CC0604F002343F2FB
:1087B0000C0E634501DB0A24A0E757F8049BBEF8C2
:1087C0000080C14500F0C1820133F2E794F87C30AB
:1087D000002BF0D0B668D4F880309E42EBD894F8E5
:1087E000E830002BE7D1524B0360202343604E4B0F
:1087F000052001F050FA0028DDD194F8E9604D4FD2
:108800004D493246384604F022FE4C4B464A4C490C
:108810000420C3E9007601F025FA00287FF449AF6F
:10882000484B94F8A1201860032AC4D8DFE802F06E
:108830000C3B2D4294F87C30002BBCD0F668D4F869
:1088400080309E42CBD3B6E794F8B020002AB2D055
:10885000D4F8B4201A603C4A354E02F12007106863
:108860005168344603C40832BA422646F7D1186824
:1088700000283FF457AF354A002102F0C1FF80B90C
:10888000012402F0FFFD2C7038E794F8A820002A9C
:1088900091D0D4F8AC1019602D4AC2F5FC22914257
:1088A000D9D904242AE794F8A220002A83D0D4F846
:1088B000A420CFE794F8A820002A3FF47CAF94F8D6
:1088C000A220002A3FF477AFD4F8A420D4F8AC104B
:1088D00050181860002A3FF425AF0029DCD121E7A9
:1088E0001B78002B7FF467AFE3E60D4B1A6CB26088
:1088F000DB6B73604FF480733360FEE6013B052B46
:1089000000F22182DFE813F02600680031012C011B
:108910001F021702602C0020E830002038360020AB
:1089200000360020EC300020CC2C00207C310020D0
:10893000AC2C002018320020D6310020A42C0020BE
:1089400004D60700DC300020A7310020E0300020F2
:1089500000800700AB68002B3FF4E4AEC3F30B02CA
:108960003AB1A84AA849526D09681A448A427FF46C
:10897000D9AEB3F5805F94D8A44A12780AB9082416
:10898000BCE6A04AA049506D096803448B42F6D862
:10899000D36C9364AB685364106510639C4A9D4C20
:1089A0001378A968013303F0030313709A4B002274
:1089B0001A802368994A01332360994B1B6801F69A
:1089C000FF71090B184402F06BFC00283FF495AED0
:1089D0002368013B23606CE68A4C236D7360A36CB3
:1089E000B3608A4B1B78002BC9D0A968B1F5807F92
:1089F0003FF657AFD4E914329B1A626C0B44934292
:108A00003FF690AE04F148026868834FDFF80082B9
:108A1000DFF810A200F048FFA064AA68236D134499
:108A200023657360A36CB360AA683B889918FF291B
:108A3000696839D898F80000019303EB002050448E
:108A400004F005FDA868019B184438803A88002A84
:108A50003FF453AE636D206B616CD31A03448B42B9
:108A6000FFF44BAE6E4B6B4DD3F800C02B6898F8FB
:108A700000E06C49013303322B609208674B01EB35
:108A80000E21604402F0C4FB00285ED1236B3A88BB
:108A90001344236398F80030013303F0030388F88C
:108AA000003000233B8028E698F80090C3F5807BD7
:108AB0004FEA09291FFA8BFB09EB03005A46504481
:108AC00004F0C5FC4FF480733B80AB68A3EB0B0351
:108AD000AB606B685B446B60DFF838B1504B206B68
:108AE000D3F800C0DBF800300133CBF8003040226F
:108AF0004A4B0AEB0901604402F08AFBC0B9236BC0
:108B00003A881344236398F80030002201333A80F6
:108B1000AA6803F0030388F80030002A96D0414881
:108B2000696800EB032004F092FCAB683B808DE7A2
:108B3000DBF80030013BCBF80030E36CA364636DDD
:108B400023657360E36CB360DDE72B68013B2B604A
:108B5000E36CA364636D23657360E36CB36099E7B2
:108B6000284B1A6D72609B6CD0E5264DD5E9142315
:108B7000696CD31A99427FF402AFAB6C6A6500202E
:108B8000EB64686402F07EFC1F4B296D1A68914209
:108B900098467FF4B2AD1F4C2368002B4CD1224E77
:108BA00096F8B930032B4AD1204F1D49204B3B602A
:108BB0004FF020093B46D8F800200968C7F8049018
:108BC000052001F068F84A46002806F1BB01386824
:108BD00014BF0A24012404F02CFC002818BF05242B
:108BE0006B6973B3012B7FF4E6AD124B012C40F09F
:108BF0009E8096F8A120032A00F29780DFE802F019
:108C00002383898F00360020DC300020E8300020EC
:108C1000D42C0020E4300020D830002075850700D7
:108C2000E0300020D82C0020EC300020CC2C00209C
:108C3000AC2C00202436002002F07CFAACE70A2499
:108C4000CEE74A4BD2E701229A60D6F88020AA608C
:108C5000AA6C5A60D8F800201A60002120224448EB
:108C6000444E454FFFF75EFCB222FF214348FFF719
:108C700059FC00232B63424D284602F003FC1128C7
:108C80007FF43CAD32683F4B00BF00BF00BF00BF68
:108C900000BF00BF00BF00BFBA422FD000BF00BF5F
:108CA00000BF00BF00BF00BF00BF00BF00BF00BFCC
:108CB00000BF00BF00BF00BF00BF00BF00BF00BFBC
:108CC00000BF00BF00BF00BF00BF00BF00BF00BFAC
:108CD00000BF00BF00BF00BF00BF00BF00BF00BF9C
:108CE00000BF00BF00BF00BF00BF00BF00BF00BF8C
:108CF00000BF00BF00BF00BF00BF00BF013BC3D12A
:108D000002F018FAB8E7A5229A60D6F8A4206A63A0
:108D10009EE7AA229A60D6F88020EA6098E7AC2203
:108D20009A60D6F8A4206A63F5E70A2490E7002247
:108D3000C3E9012290E7144B9A6CB2601B6D73601B
:108D40004FF48053D8E50224D8E494F8A130032BE3
:108D50003FF631AD01A757F823F000BFCD870700DC
:108D6000DF870700358807003588070018360020A0
:108D700038360020642C00200024F4005C360020EB
:108D8000D5850700A0860100003600207047704797
:108D9000BFF34F8F0549064BCA6802F4E0621343E4
:108DA000CB60BFF34F8F00BFFDE700BF00ED00E0D9
:108DB0000400FA054FF0A043D3F81005054B93F8D3
:108DC000972093F89630D040DB0648BFC04300F0B0
:108DD000010070477CD6070008B5FFF7D9FF08B53A
:108DE000FFF7D6FF0D4B00EB80001A1870B51B5C27
:108DF0005478C3F300134FF0A04204F5E0758B42A2
:108E00004FF003064FF0010342F8256003FA04F324
:108E10000CBFC2F80C35C2F8083570BD7CD607000F
:108E2000022808B50BD003280BD078B90848FFF703
:108E3000AEFF01210C20BDE80840FFF7D3BF054875
:108E4000F5E70548BDE80840FFF7A1BF08BD00BF32
:108E50000CD6070021D607001ED607002DE9F843DF
:108E6000FFF7A8FF0546E8B1FFF790FF39483A4FF2
:108E7000DFF8F480DFF8F490FFF789FF3748FFF759
:108E800086FF3748FFF783FF40F6B834FFF792FFBD
:108E90000646002857D044B9264601210C20FFF78A
:108EA000A1FF35462846BDE8F8833A6840F2E7332B
:108EB00000BF00BF00BF00BF00BF00BF00BF00BFBA
:108EC00042452FD000BF00BF00BF00BF00BF00BFA2
:108ED00000BF00BF00BF00BF00BF00BF00BF00BF9A
:108EE00000BF00BF00BF00BF00BF00BF00BF00BF8A
:108EF00000BF00BF00BF00BF00BF00BF00BF00BF7A
:108F000000BF00BF00BF00BF00BF00BF00BF00BF69
:108F100000BF00BF00BF00BF00BF00BF00BF00BF59
:108F200000BF00BF013BC3D114F0030F0CBF0121F0
:108F300000210C20FFF756FF630602D14846FFF7D9
:108F400026FF013CA2E7002CA7D00648FFF71FFF31
:108F50002E46A2E72DD60700642C00203AD6070043
:108F600051D607006CD607000024F4006AD607002B
:108F7000002110B50C20FFF735FF104B93F8972018
:108F800093F89630DB0647BF03210B4602230121ED
:108F90001B0443EA810302F5E0724FF0A04141F85F
:108FA000223002F08DF8044608B1FFF7F1FE43F2DB
:108FB0000803186802F0A8F8204610BD7CD6070008
:108FC00030B54C1CE40012F00303A4B20ED1084DDE
:108FD0002A602244074C2260074A1370074A137024
:108FE000074A1080074A1846118030BD0720FCE769
:108FF000703200206C32002068320020783200206D
:1090000074320020763200202DE9F743294D2B8859
:109010008B4206460C46174647D34FF000080DF129
:1090200007008DF8078000F005FC234B234A1878D1
:109030001178CBB2224909888B4238BF0133C0B2C4
:1090400038BF5FFA83F8404528D092F80080137843
:10905000DBB2994286BF0133DBB2002313709DF867
:10906000070000F00BFC4FF6FF7398451FD0154B1F
:109070001B6803EBC80943F8387096B18CB1124BEA
:1090800028881B682246314608FB003004F0DFF9CF
:10909000A9F80440002003B0BDE8F0834FF6FF7844
:1090A000DDE70020A9F80400F5E70920F3E7042034
:1090B000F1E700BF743200207832002068320020CF
:1090C00076320020703200206C320020F8B5124C4D
:1090D000124D264622782B789A4200D1F8BD23788B
:1090E0000F48104A078812680F48DBB219B202EB2A
:1090F000C10C006852F83120BCF8041003FB0700D3
:1091000090470A4A23781288DBB29A4286BF01331D
:10911000DBB200233370DDE77832002068320020B4
:1091200074320020703200206C3200207632002031
:1091300010B50A494A788C78531CDBB29C4208BFB0
:1091400000230C789C421FBF0370486802EB420268
:1091500000EBC20008BF002010BD00BF803200201D
:1091600073B5054600240DF107000E468DF8074043
:1091700000F060FB0DF10600FFF7DAFF90B106701A
:10918000094B9DF8062045605A709DF8070000F0D5
:1091900075FB24B9054B4FF48012C3F8002120461B
:1091A00002B070BD0424F0E78032002000E100E04E
:1091B000204B21491A682F2300BF00BF00BF00BF0A
:1091C00000BF00BF00BF00BF8A422FD000BF00BF5A
:1091D00000BF00BF00BF00BF00BF00BF00BF00BF97
:1091E00000BF00BF00BF00BF00BF00BF00BF00BF87
:1091F00000BF00BF00BF00BF00BF00BF00BF00BF77
:1092000000BF00BF00BF00BF00BF00BF00BF00BF66
:1092100000BF00BF00BF00BF00BF00BF00BF00BF56
:1092200000BF00BF00BF00BF00BF00BF013BC3D1F4
:10923000704700BF642C00200024F4000C4B0D4844
:109240004FF4003210B5C3F8802001244FF480336E
:10925000C0F84833C0F808334460FFF7A9FF064B55
:10926000846000201860FFF7A3FF044B187010BD46
:1092700000E100E000100140983200208932002017
:109280002DE9F8432649274B0025C1F84051C1F884
:109290004451C1F84851C1F84C51C1F80051C1F8CE
:1092A00004511B68002B34D0D1F804451E49DFF867
:1092B0008C800968641A24F07F442F461A68A24201
:1092C00012D8A41A15441A7CDE6962B1D8F800904D
:1092D0001F74D3E90521B9F1000F1ED01046C8470D
:1092E00008B1FFF77CFDB6B9104A114B11781B7815
:1092F0008B4205D10133DBB2022B08BF0023137070
:1093000012780C4B43F822500B4B4FF48012C3F8E9
:109310000021BDE8F8833346D0E708469047E2E7EE
:10932000001001409C32002098320020953200202D
:10933000943200208C32002000E100E07C320020DA
:109340002DE9F04FB04AB14813780078B0499842FF
:1093500087B0D1F800C000F0AC800133DBB2022B43
:1093600008BF002313701278AA4B53F822400CEB6D
:10937000040323F07F430B6001230193A64AA7480F
:109380001378D0F800E050780390506892780492F7
:10939000A34A02900020D1F800A092F8009019464C
:1093A00072468046039DA94240F08680B8F1000FC6
:1093B00005D09B4981F800909549C1F800A09749D4
:1093C00000B10A6001980A68002840F0C780BEEB2F
:1093D000020218BF0122019200260A680592904AF3
:1093E000059992F800B08A4A4FF0000ED2F800A01A
:1093F0007746F046002E40F0B680039A9A4240F03D
:10940000D2800FB1844B1A70844BBEF1000F00D094
:1094100019601B68059A9A4202D1019A002A42D02B
:10942000002B00F02681D3F800907E4C784BD4F8C6
:10943000046518687C4F351A3B7825F07F45033565
:109440009BB94FF48033C4F84433C4F80433774BEA
:109450004FF400324FF00108C3F880211A60C4F8BD
:109460000080FFF7A5FE87F80080A9452CBF48447F
:10947000401920F07F40C4F84005D4F804359B1B08
:1094800023F07F43801B033320F07F4083420AD9BF
:10949000D4F80435C4F84035FFF78AFE634B4FF427
:1094A0000032C3F800215E4B00221A7007B0BDE8FD
:1094B000F08F0024019461E701EB4106049D029FB7
:1094C0000131C9B2A94208BF0021029D07EBC607BE
:1094D00015F83660022E0BD0032E7FF463AF002AFE
:1094E0003FF460AF4FF000001074D2690120F6E73E
:1094F000D7F804B016461746002E3FF453AFB345D5
:1095000000F0BA803746F669F6E70120C1E0D2F8EC
:1095100000E0A64505D907B10A60AEEB040414606B
:109520005BE7A4EB0E047044D2F80CE0C2F80080B4
:10953000D2F81C90BEF1000F07D00CEB000727F00B
:109540007F47C2E9017ED6611646019F4A46002A3E
:10955000DDD1002F3FF441AF0A603EE700273E46D1
:109560003846B846F3E73246F6695068304DD2F8CF
:1095700008C0A0EB0A0424F07F44AC4238D864440D
:1095800014604FF00100C2E901881074C2F81C8019
:1095900031B114680868844266D8041B0C60D1613C
:1095A0004FF0010E5EE003EB4302049C029801338E
:1095B000DBB29C4208BF0023029C14F83240012C0D
:1095C00000EBC20053D14268177C002F7FF415AF27
:1095D00085685560C56895600569D560406990618A
:1095E000BBF1000F02D057605F46BEE72746BCE7DD
:1095F000AAEB000020F07F4060453ABFACEB0000D2
:109600001060C2F80080BCE7943200209532002040
:10961000983200208C320020803200209C320020C2
:1096200088320020001001408932002000E100E073
:10963000FEFF7F00A4EB0C04D0F81CC08146BCF1F7
:10964000000F0AD06046D0F800C0A445F2D3ACEBBE
:10965000040CC0F800C0844648461460C2F81CC020
:10966000C2610A461146C5E689460846EBE701276E
:10967000C3E6FFF7E3FD16E7BE420AD1D269002A2E
:109680007FF443AF08480125856092462846A846E6
:10969000A946D6F800B0F669FE61002E3FF482AE0E
:1096A00037685F4437607DE6001001402DE9F041E6
:1096B00012F0030406460F461546984627D132B3EA
:1096C000FFF7BCFD134B144A1C809F705D60134B69
:1096D000C2F800801C60124B1C70124B1C70124BA5
:1096E0004FF48012E021C3F8802183F814131A602C
:1096F00002F18042A2F56F222046C2F8086583F885
:1097000011130A4BD2F804251A60BDE8F081072036
:10971000FBE700BF803200207C3200209C3200201A
:10972000943200209532002000E100E098320020C1
:10973000074B5B684BB132B128B10368187C20B984
:1097400059745A617047072070470820704700BF5E
:10975000803200202DE9F7431E4F7B6805460E46F8
:109760009046A3B398B304292FD943697BB3437CB4
:109770000024012B0DF107000CBF8946A1468DF88E
:10978000074000F057F80DF10600FFF7D1FCD0B10B
:1097900001230370104B4560D3F80435C0E90498E9
:1097A000C0E902369DF806307B709DF8070000F096
:1097B00065F824B9094B4FF48012C3F80021204604
:1097C00003B0BDE8F0830424EFE70724F7E708249B
:1097D000F5E700BF803200200010014000E100E00A
:1097E000064A52683AB130B1426922B1002202748D
:1097F0000221FFF7B5BC0820704700BF803200206F
:10980000082910B5044602D00020FFF7E8FAD4E991
:109810000030BDE81040184707B5054ACDE9000102
:1098200008216846FFF7F0FB03B05DF804FB00BFBA
:109830000198070070B5EFF3108672B60C4A946871
:1098400001239CB993600B4B0B4DD3F8801029403A
:109850001160C3F88050D3F8841051604FF0FF328C
:10986000C3F88420047006B962B670BD0370FAE7CD
:10987000A032002000E100E0FC06FFBC10B5084B60
:109880009A685AB150B9EFF3108172B6054A1C6854
:1098900014605C685460986001B962B610BD00BF86
:1098A000A032002000E100E030B53AB11368DB439C
:1098B0000A4D0144884204D1D84330BD4FF0FF33F4
:1098C000F6E710F8012B5340082213F0010418BFEB
:1098D0002C46013A84EA5303F7D1EBE72083B8ED35
:1098E000F7B50D4617461E460446A0B199B193B18F
:1098F0000B4303439B0710D103F03EFC334600901B
:109900003A462946204603F03BFC002814BF0020BD
:109910000B2003B0F0BD0E20FBE71020F9E729DF94
:10992000704728DF70470000084B5A6E013A5A66AC
:1099300022B907490A7822F002020A701A6E01322F
:10994000042A08BF00221A66704700BFB032002008
:10995000AC32002010B50C494A6E042A044611D0DE
:109960000B6E1344032B02F101024A6688BF043BCD
:10997000182202FB031318460021FEF7D3FD2060D6
:10998000012010BD0020FCE7B032002030B50446B5
:1099900085B00D46102200216846FEF7C3FD237AEC
:1099A000012B0AD0022B0ED063680193236829464D
:1099B0009B686846984705B030BD23690293A38A27
:1099C000ADF80C30F0E70123A2898DF80030E3896F
:1099D000ADF80A20D31AADF80830E5E738B51C4BCE
:1099E0005A6E19465AB31C6E182202FB04331A7AB7
:1099F000012A07D0022A23D018460921BDE83840A1
:109A0000FFF7C4BF1825D88A9A8A05FB0414D4E945
:109A10000314121AB2F5806F4FEA80000144B4BFFC
:109A200092B24FF480622044FFF779FF11280BD1E6
:109A3000084A137823F0020343F00403137038BD7F
:109A40009889FFF76EFFF1E70028F8D0D4E700BF50
:109A5000B0320020AC320020054A137813F0060F14
:109A600004D143F002031370FFF7B8BF704700BF83
:109A7000AC320020034A137843F001031370002036
:109A8000704700BFAC320020F7B51E461E4B1B7856
:109A90001746DA0704460D4628D548B31B4B9842B3
:109AA00026D31B4B984223D227B319B347EA0103AD
:109AB0009B0721D103688B4220D8426801EB8603C3
:109AC0009A421BD3E6B101A8FFF744FFD0B1019B36
:109AD000089AC3E90042019901230B72C1E9037599
:109AE0008E82FFF7B9FF002003B0F0BD0120FBE735
:109AF0000220F9E70320F7E70620F5E70520F3E762
:109B00000420F1E70720EFE7AC320020702C0020A2
:109B1000802C0020F7B51F461D4B1B78DB07054640
:109B20000C46164625D530B31A4B984223D31A4B10
:109B3000984220D209B3C1F30B0303BB03688B42E5
:109B40001FD8436801EB023293421AD3DEB101A859
:109B5000FFF700FFC8B1019AC2E90057019B02223A
:109B6000240B1A729C811E82FFF776FF002003B03F
:109B7000F0BD0120FBE70220F9E70320F7E706200C
:109B8000F5E70520F3E70420F1E70720EFE700BF42
:109B9000AC320020702C0020802C002038B52A4ADE
:109BA00013780146980742D5284A146E18200229D6
:109BB00000FB042005D003292DD0BDE83840FFF775
:109BC0000DBF234B00211970037A012B0CD0022BFF
:109BD000F3D18389028A01338381C38901339BB224
:109BE0009A42C381E9D111E0858AC38AE91AB1F5A5
:109BF000806FB4BF89B24FF480610B4418219BB2CF
:109C000001FB04229D42D382D7D10021FFF7BEFE83
:109C1000FFF78AFED1E70E4A13780133DBB2032B3C
:109C200001D81370C9E7002313700821EEE7590724
:109C3000C3D50649496E03F0FB0313700029BCD05D
:109C400043F00203EDE700BFAC320020B032002049
:109C500018330020024B586E031F5842584170477A
:109C6000B0320020042810B40C4611460DD16268B1
:109C7000402A0ED15A68402A0BD120681B685DF833
:109C8000044BD1E90012FFF72BBE06205DF8044B10
:109C900070470920FAE7F0B505289DB00E46174633
:109CA0001C4615D15D68202D14D1684600F0B2F82D
:109CB00060B93A463146684600F0DCF830B9012216
:109CC0002168684600F0FAF800B965601DB0F0BD83
:109CD0000620FBE70920F9E72DE9F04FC9B008AAF3
:109CE00001F1400514464B780E781B0443EA0663E5
:109CF000CE7833438E78043143EA06238D4244F80C
:109D0000043BF0D11024916B16464FEAF14383EAED
:109D1000714383EA9123716A366852F8045F3144D3
:109D20000B444FEAB54181EAF51181EAD5010134CE
:109D30000B44402CD363E6D1D0E914E30093836D48
:109D40000193C36D0293036E0393436E0493836E7A
:109D50000593C36E0693DDE9057BDDE9031CDDE9B0
:109D600001592B4B009E079374464FF00008079B48
:109D700053F8042B07934FEAF12383EAB11383EAE4
:109D8000716A08AB53F828301A440AEB020327EA39
:109D9000010A01EA0C028AEA02021A444FEA743A02
:109DA00086EA05035A448AEAB40A06EA050B234008
:109DB00083EA0B038AEAB45A08F101089A44B8F11D
:109DC000400F02EB0903BB465244A94619D1724425
:109DD0000265009A22444265019A32448265029AE1
:109DE0002A44C265039A1A44049B02660B444366E4
:109DF000059B63448366069B3B44C36649B0BDE84C
:109E0000F08F674635468C46264619461446AEE71F
:109E10001CD7070030B5E0B10F4A104900240025D7
:109E2000C0E91245C0E914120D4C0E4A0E4DC0E9AE
:109E300016420E4AC0E918520D4A826602F1745267
:109E4000A2F523020023A2F692420364C2661846DA
:109E500030BD0E20FCE700BF85AE67BB67E6096A30
:109E600072F36E3C3AF54FA57F520E518C68059BFC
:109E7000ABD9831FF8B50446F0B10AB90020F8BD8C
:109E8000D1B10D468E180027B542F7D0236C15F8D6
:109E9000012BE2540133402B2364F5D121462046A7
:109EA000FFF71AFFD4E9123113F5007341F10001F5
:109EB000C4E912312764E7E70E20E0E770B50D46EC
:109EC00016460446002877D0002975D0026C802100
:109ED000372A02F1010381544FF0000242D8382B97
:109EE0003BD1D4E91223206C0821E1FB002310466A
:109EF00012BAE2631A0A194684F83B3084F83A2011
:109F00001A0C1B0EC4E9120184F83920214684F88A
:109F100038302046FFF7E0FE691E76B30023E26E7C
:109F2000DA4001F8012FA26EDA400A71626EDA405F
:109F30000A72226EDA400A73E26DDA400A74A26D88
:109F4000DA400A75626DDA400A76226DDA4008332B
:109F5000202B0A77E3D1002070BDE2540133BEE725
:109F6000E25401333F2BFBD921462046FFF7B4FED4
:109F700038220021FEF7D6FAB3E71823226DDA4023
:109F800001F8012F626DDA400A71A26DDA400A729F
:109F9000E26DDA400A73226EDA400A74626EDA40C9
:109FA0000A75A26EDA400A76E26EDA40083B13F1D7
:109FB000080F0A77E2D1CEE70E20CDE70368D3E998
:109FC00000329A422FBFD01A80680130801838BF03
:109FD000C01A704702688168536810688B4234BFAA
:109FE00001330023C31A584258417047F7B5002384
:109FF00004460DF107000D468DF80730FFF71AFCF7
:10A000002046FFF7E7FF10B1237C002B3CD12268EC
:10A01000A16853688B4234BF591C0021516038B18C
:10A020002168A0680A68824234BF013200220A60B7
:10A03000E2686068511E072920D8DFE801F00410AB
:10A040001F141F1F1F182A78C2542046FFF7B6FF9F
:10A0500023689A68824200D29860002415E02A881A
:10A0600020F81320F1E72A6840F82320EDE7D5E92E
:10A07000006700EBC300C0E90067E6E7294603FB81
:10A08000020003F0E4F9E0E704249DF80700FFF77D
:10A09000F5FB204603B0F0BD13B500230DF102001F
:10A0A0008DF80230FFF7C6FB00F074FFE8B9124BE1
:10A0B0001A68D2B1114CD4F80823D20715D518600C
:10A0C0001B680193019B0E48D4F808358DF80330C6
:10A0D0000DF10301FFF78AFF0948FFF77BFF20B16D
:10A0E000084A0123C4F8083313609DF80200FFF703
:10A0F000C5FB02B010BD00BF00D1004000D0004041
:10A100001CD8070004D000400B4B0222C3F80425E2
:10A11000D3F80024002AFBD0C3F80805D3F80024A4
:10A12000002AFBD00022C3F80425034AD2F80034E9
:10A13000002BFBD0704700BF00E001400F4B30B553
:10A140000124C3F80445D3F80044002CFBD00B4B8A
:10A1500001EB8202401A914207D10022C3F8042584
:10A16000D3F80024002AFBD030BD441851F8045B1A
:10A170002560D3F80044002CFBD0ECE700E0014060
:10A180006CDF70476DDF704772DF704773DF7047B9
:10A1900074DF704776DF70477ADF70477CDF704787
:10A1A0007DDF70477FDF704786DF7047A0DF704735
:10A1B000A2DF7047A5DF7047A6DF7047A8DF7047B2
:10A1C000A9DF7047ADDF704763DF704767DF704717
:10A1D00013DF70477FB50023CDF80A30ADF80E309D
:10A1E00001238DF80A300DF10603ADF80810049331
:10A1F00002A9044BADF806200593FFF7DDFF07B079
:10A200005DF804FBB0330020FEF7E9BD10B40D4B40
:10A21000024618884FF6FF7398420FD00A4B1B680E
:10A22000DB070BD5094B60245A7099701C70084BE2
:10A230005DF8044B99890322FFF7CCBF08205DF835
:10A24000044B7047622C0020AC330020B033002058
:10A250009833002010B5314C23685A075CD443F082
:10A26000040222602E4A2F4811682F4A00BF00BF07
:10A2700000BF00BF00BF00BF00BF00BF81422FD0A2
:10A2800000BF00BF00BF00BF00BF00BF00BF00BFD6
:10A2900000BF00BF00BF00BF00BF00BF00BF00BFC6
:10A2A00000BF00BF00BF00BF00BF00BF00BF00BFB6
:10A2B00000BF00BF00BF00BF00BF00BF00BF00BFA6
:10A2C00000BF00BF00BF00BF00BF00BF00BF00BF96
:10A2D00000BF00BF00BF00BF00BF00BF00BF00BF86
:10A2E000013AC3D1114A10884FF6FF72904204D050
:10A2F0001321FFF74FFF68B110BD9B070AD5FFF789
:10A3000047FF0028F8D10120FEF78AFD236843F0BB
:10A310000203236000F0F8FB0020EDE7AC330020DF
:10A32000642C00200024F400C0D40100622C002022
:10A3300030B52A4D296811F002018BB04BD11022A3
:10A3400001A8FEF7EFF80B23ADF80230244B05937C
:10A3500045F60213ADF818300DF10201FE230DF1A0
:10A360001D008DF81A30FFF71BFF044640BBBDF8F7
:10A3700002100B2927D84B1C8DF81B3009231944D8
:10A380008DF81C3089B200231A46C9B205A8FFF720
:10A39000FBFE0446A0B98DF8040002908DF80C0075
:10A3A0002823ADF8100001A8ADF80E30FFF7EEFE3F
:10A3B000044628B9FEF734FD2B6843F002032B60F6
:10A3C00020460BB030BD0C238DF81B3008238DF8D0
:10A3D0001C301421D7E70024F2E700BFAC33002083
:10A3E0000201060310B4154B024618884FF6FF739E
:10A3F00098421FD0124B1B68DB071BD5114B602402
:10A400001C7003245C7001249C70140ADA701C71A7
:10A41000140C120E9A710A0AD9711A720A0C090EDA
:10A420005A7299725C71084B5DF8044B99890B2242
:10A43000FFF7D0BE08205DF8044B7047622C002067
:10A44000AC330020B0330020983300202DE9F041D8
:10A45000044688B000F05EFB2388142B00F0408196
:10A4600018D8102B71D005D8022B00F08A8008B0C4
:10A47000BDE8F081112B77D0132BF8D1B44800231D
:10A480001A4685210088FFF78DFE0028EFD0FEF7E1
:10A49000A6FCECE7522B00F02A8148D8502B00F0A4
:10A4A0002D81512BE3D1A579002DE0D01022002180
:10A4B0000DEB0200FEF736F8022DD8D1A54D22890A
:10A4C000AB899A42D3D1A37B043B022BCFD99DF811
:10A4D00016309F4E298A3088CDF808D043F001030A
:10A4E0008DF81630238AADF81830638AADF81A302B
:10A4F000022204F114038DF810200793ADF8042014
:10A50000002301AAADF80630FFF754FEB04600283C
:10A510003DD1684600F056FB002838D140F2FD13CB
:10A5200004A93088ADF81430FFF748FE9FE7552B9B
:10A5300000F01A81562B9AD1A379002B97D1844B26
:10A5400013211888FFF726FE9FE70120FEF768FC1D
:10A550000220FEF765FC7E4BA2881A807E4A1368B3
:10A5600023F00203136082E70320FEF759FCFFF794
:10A57000DFFE08B1FEF733FC754B4FF6FF721A8011
:10A5800075E7734B00211888FFF720FE7DE7002355
:10A5900004A9B8F80000ADF81430FFF70FFE00284A
:10A5A0007FF465AFCDE904000690CDE9010003908A
:10A5B000207D431E052B00F29180DFE803F0032984
:10A5C000391E8F4C638A062B04D003210120FFF72C
:10A5D0001DFE4CE7614B1A88614B1A80637D029324
:10A5E00001A9D4F816300393012404AA00208DF8A1
:10A5F0000440FEF749F80146E8E7032301A904AA4D
:10A6000000208DF80430FEF73FF801460420DEE715
:10A61000638A032B02D003210220D8E7A27D637D49
:10A6200043EA02234D4A13804D4A01211380F3E788
:10A6300004230DEB030104AA00208DF80430FEF77B
:10A6400023F80128014604D1DDE90501FFF7CAFE20
:10A650000DE70320BBE7638A022B02D0032106200B
:10A66000B5E7637D029301A9062704AA00208DF8AF
:10A670000470FEF709F801280146F0D1B8F800008F
:10A680004FF6FF7398423FF4F2AE334B1B68DB0783
:10A690007FF5EDAEDDE90464324B069A9970310A1C
:10A6A0001971310C5971210A1972210C5972110A50
:10A6B000DE70DC71360E240EDA721973110C120E74
:10A6C0004FF0600C59739A739E719C720F22A98986
:10A6D00083F800C05F70FFF77DFDC8E6032176E7D1
:10A6E00000231A461946A088FFF75EFDCDE6002339
:10A6F0001A461946A088FFF763FDC6E6154BE288A7
:10A700009B889A427FF4B3AE0020022301908DF81B
:10A71000043004F11203029304AA238A039301A9CB
:10A72000CDE904000690FDF7AFFF0C4B1D88002D0E
:10A730003FF49DAE0A4C2388013B9BB22380002B43
:10A740007FF495AEDDE90501FFF74CFE25808EE62E
:10A75000622C002098330020AC330020C03300204E
:10A76000C2330020B03300201721A088FFF72AFD54
:10A770008BE600BF2DE9F043054695B0002800F0B8
:10A780008E80484B4FF6FF721A8001204FF65963B6
:10A790002A4602A98DF80A00ADF80830FFF706FD39
:10A7A0000446002877D1404B04AA03F1100716464F
:10A7B00018685968144603C40833BB422246F7D1CF
:10A7C000A91C3046FFF700FD0446002863D101466E
:10A7D0001C220DA8FDF7A6FE9DF83430ADF804400C
:10A7E00043F004038DF83430AB788DF80E3002233B
:10A7F000ADF80C301423CDE90A44ADF82C302B46CB
:10A800000C94A04604F0F80444F0030401AE4FF0A9
:10A81000110903AF33F8040B8DF8064008AA0DA9FF
:10A820008DF80590CDE90876FFF7C2FC044690BB91
:10A8300001461C220DA8FDF775FE9DF83430ADF8D9
:10A84000044023F0180343F018038DF83430AB783C
:10A850008DF80E300123ADF80C301723CDE90A44F2
:10A86000ADF82C302B4608F0E80848F0130833F810
:10A870000C0B0C9408AA0DA98DF805908DF8068094
:10A88000CDE90876FFF794FC044620B9074A13681F
:10A8900043F001031360204615B0BDE8F0830E2499
:10A8A000F9E700BF622C002030D80700AC3300204D
:10A8B00000B5344B8BB01868019000F062FD0028A1
:10A8C0005CD13148FFF784FC002857D12F4B304929
:10A8D000502201A800F064FB08B1FEF780FA0121C4
:10A8E00003AA084600F0B4FB002847D1172303A8A9
:10A8F000ADF81C3000F0C4FB00283FD1254800F023
:10A9000081FB00283AD1CDE90300112301A88DF87D
:10A910000030FFF737FC88BB9DF8053001A80133F4
:10A920008DF80530FFF72CFC40BB07221A4968461A
:10A93000FFF734FC10BB19494FF0C87303A8CDE9E9
:10A940000313FFF729FCC8B91548FFF713FFA8B98F
:10A950001822014603A8FDF7E5FD4FF4804340F6B9
:10A96000CD42CDE9042303238DF8183003A80D4B05
:10A97000099300F093F808B9FFF7DAFC0BB05DF823
:10A9800004FB00BF40D8070000800700B1B00700FB
:10A99000483300204DA4070044D807000C001800DD
:10A9A0009833002009A2070075DF704776DF7047F3
:10A9B0007ADF70477BDF704737B5164B18884FF644
:10A9C000FF73984210D0144A144D1378297B013339
:10A9D000DBB2994213702C4608D31149FFF7E4FF0C
:10A9E00010B1AB6903B1984703B030BD00231370B9
:10A9F0002B7C33B13B21FFF7D9FF10B1AB6903B119
:10AA000098476369002BEFD000228DF8042001A83D
:10AA1000E9E700BFC633002014340020C83300200B
:10AA20000C34002037B5174B174A5B881188174C38
:10AA3000174D994208D852889A4205D36369F3B9F1
:10AA400000232B7003B030BD2A783AB16369002B24
:10AA5000F6D000228DF8042001A80EE00D48D4E9BC
:10AA600001130078002818BF19460B48FEF772FE44
:10AA70000028E5D0A369002BE2D09847E0E7012247
:10AA8000E8E700BF043400200C340020C833002065
:10AA9000C433002014340020E433002070B5054690
:10AAA00006460FCD114C0FC495E80700104B84E803
:10AAB000070000221A7032680E489AB113680360CA
:10AAC00053684360FFF774FF78B90B4B0B484FF6A0
:10AAD000FF721A800A4B0B4A00211970BDE87040C2
:10AAE000FEF726BEFFF766FFEEE770BDC833002015
:10AAF000C43300200C340020C63300204CD807009B
:10AB000014340020B9A907000148FEF769BE00BF50
:10AB1000E433002010B50388112B2ED002D8102B5F
:10AB200017D010BD122B3BD0502BFAD1204CC2882D
:10AB3000E3899A42F5D1038A022BF2D1123000F058
:10AB400041F8B0B91B48FEF74BFE0028E9D0A369D5
:10AB500021E0194B82881A8000F1100303CB174AB9
:10AB6000174B1060516000221A70114BDB89002BCB
:10AB7000D7D1BDE81040FFF755BF0F4B0D484FF63A
:10AB8000FF721A800E4B00221A70FEF729FE002871
:10AB9000C7D0074B9B69002BC3D0BDE810401847B6
:10ABA00000F1080303CB054A10605160E1E700BFE4
:10ABB000C8330020E4330020C633002004340020D2
:10ABC00014340020007800F001007047BFF34F8F6D
:10ABD0000549064BCA6802F4E0621343CB60BFF339
:10ABE0004F8F00BFFDE700BF00ED00E00400FA0555
:10ABF000094B1B78062B0CD1084B1B681A0708D190
:10AC0000074B186800F0F000A0F13003584258419B
:10AC100070470020704700BFE00F00F0E40F00F025
:10AC2000E80F00F00C4B1B78062B10D10B4B1B6868
:10AC30001A070CD10A4B186800F0F003302B08D02B
:10AC400000F0E000A0F14003584258417047002056
:10AC500070470120704700BFE00F00F0E40F00F0E4
:10AC6000E80F00F008B5FFF7C3FF10B1774B784A43
:10AC70001A60FFF7D7FF28B1764B774A1B68C3F3FA
:10AC800042331360FFF7B4FF20B1744AD36823F056
:10AC90008073D360FFF7C6FF40B14FF080430022BE
:10ACA000C3F80C21C3F81021C3F83825FFF7A0FF23
:10ACB00010B16B4B03221A60FFF79AFF40B1694B4A
:10ACC00005221A6001229A6700229A603F225A6088
:10ACD000654B1B78062B50D1644B1B6819074CD170
:10ACE000634B1B6803F0F003502B46D14FF08052AA
:10ACF000604BD2F80414C3F82015D2F80814C3F836
:10AD00002415D2F80C14C3F82815D2F81014C3F87F
:10AD10002C15D2F81414C3F83015D2F81814C3F84F
:10AD20003415D2F81C14C3F84015D2F82014C3F817
:10AD30004415D2F82414C3F84815D2F82814C3F8DF
:10AD40004C15D2F82C14C3F85015D2F83014C3F8AF
:10AD50005415D2F83414C3F86015D2F83814C3F877
:10AD60006415D2F83C14C3F86815D2F84014C3F83F
:10AD70006C15D2F84424C3F87025FFF753FF28B1AF
:10AD80003D4B3E4A1B6803F04F0313603C4AD2F828
:10AD9000883043F47003C2F88830BFF34F8FBFF39D
:10ADA0006F8F4FF01023D3F80C22D2071ED5354BEE
:10ADB0000122C3F80425D3F80024002AFBD04FF069
:10ADC0001022D2F80C3223F00103C2F80C322D4BC2
:10ADD0001A46D3F800140029FBD00021C3F804154B
:10ADE000D2F80034002BFBD0FFF7F0FED3F800229E
:10ADF000002A03DBD3F80432002B23DA214B012293
:10AE0000C3F80425D3F80024002AFBD04FF0102209
:10AE10001521C2F80012D3F80024002AFBD04FF00D
:10AE200010231522C3F80422164B1A46D3F8001437
:10AE30000029FBD00021C3F80415D2F80034002B00
:10AE4000FBD0D1E7104B114A1A6008BD74C007400F
:10AE50000DF0ADBA440200103C050040F0ED00E0FA
:10AE6000A005004010560040E00F00F0E40F00F095
:10AE7000E80F00F000C0004058020010E40E00404F
:10AE800000ED00E000E00140642C00200090D003C1
:10AE900048DF704710DF704760DF704761DF704741
:10AEA000FDF79ABF0A4A92F816335B060CD5094B98
:10AEB000986828B11A6842F480021A60002070472E
:10AEC0004FF480031360704742F20200704700BFE6
:10AED00000E100E0A03200202DE9F347274B1B786A
:10AEE00003F0FF08002B3ED0254D264E2B6832681C
:10AEF000B3FA83F77F09002A3CD0DFF88C9099F8E9
:10AF0000003003F0FF0473BB01A8FFF7C1FF052861
:10AF100021D0E0B1FDF763FF1FBB1B4FDFF86C9042
:10AF2000DFF86CA03B78F3B9B9F80030ADF8043025
:10AF3000DAF8003001A91846FFF7B0FF052815D050
:10AF400058B1FDF74CFF002CECD12746D5E733680C
:10AF500001989847E0E74446DEE72A68184690479C
:10AF6000F1E7002CCBD002B0BDE8F087002CFAD17D
:10AF70004446EAE7002BF6D04446CEE720340020D2
:10AF800018340020243400202134002016340020FE
:10AF900028340020014B1878704700BF203400206F
:10AFA00010B509B38C071FD1104C216010490A80DD
:10AFB000104A1360104A1368C3F340331BB14FF4B7
:10AFC0000051C2F880100D49FFF764FF28B11BB192
:10AFD000094B4FF400521A6010BD094B01221A7040
:10AFE000BDE81040FFF75EBF0720F5E728340020DA
:10AFF000163400201C34002000E100E0A1AE070060
:10B000002034002018B1034B1860002070470E2038
:10B01000704700BF1834002018B1034B186000209F
:10B0200070470E20704700BF2434002008B5074B3E
:10B030001B682BB1984738B1BDE80840FDF7CFBE7B
:10B04000BDE80840FFF748BF08BD00BF1C34002022
:10B0500070B5144605460E4616220021A01CFDF7C9
:10B0600061FA00214FF00002012361F30002238006
:10B07000A16122752672657205B1A372002070BDB0
:10B0800007B5054B0193019B00936946FFF704FF49
:10B09000019B03B05DF804FB002C002008B511B142
:10B0A0000020FDF79CFEBDE80840FFF715BF00003B
:10B0B0000021024A0846FDF7A7BF00BF9DB0070068
:10B0C00008B500F039F808BD13DF7047F0B5034646
:10B0D000186880F308885868FF2464B2EFF3058588
:10B0E000002D01D1A64600472546064621273FBA36
:10B0F000F0B40024002500260027F0B4F92040B267
:10B10000004700BFF0BD00BF10B5044600F039F99C
:10B1100068B9074B4FF0FF32C3F880202046FFF795
:10B12000D3FF20B92046BDE81040FFF7CFBF10BDC8
:10B1300000E100E0FDF7CABF13B50023019300F062
:10B14000E5F901A800F09CFA08B101230193FDF78D
:10B1500085FED8B101230193154B164A0521002025
:10B16000FEF7A4FA08B1FDF73AFE134A14210820AD
:10B17000FDF726FF08B1FDF732FE00F0F1F90446B5
:10B1800098B9FDF74DFAFDF7A1FFFCE7019C002CF3
:10B19000E2D100F01BFB0028DED000F017FB20B14D
:10B1A00043F208031868FFF7AFFF204602B010BD56
:10B1B000199807007C3500202C340020074A1368BA
:10B1C00029B923F00303136043682BB1184723F018
:10B1D000010343F00203F6E7704700BFF435002097
:10B1E00008B568B1FEF746FC08B1082008BD06485E
:10B1F000FFF712FF0028F8D1044B04221A60F5E78C
:10B20000024B1860F2E700BF9D9B0700F435002059
:10B210002DE9F041DFF884801C46D8F8003013F0A7
:10B22000040F86B006460D46174616D09A0729D455
:10B2300043F00103C8F800300A4600940146BBB24F
:10B240001548FEF721FC28B9D8F8003043F0010377
:10B25000C8F8003006B0BDE8F081A9B1A0B105433F
:10B2600015F0030512D19AB1FEF768FF94B102A858
:10B2700029468DF80850CDE90346ADF81470A04773
:10B280002846E7E70A20E5E70320E3E70620E1E7B1
:10B290000420DFE72046DDE7702C0020F435002095
:10B2A0002DE9FF41224F3B680D46590706461446DB
:10B2B00015D59A0736D443F001033B600146234677
:10B2C000AAB21C48FEF726FC3B6828B123F0010314
:10B2D0003B6004B0BDE8F08143F00103F8E7C0F340
:10B2E0000B030BBB2F4680464046FEF70DFF013F88
:10B2F00008F58058F8D106EB0535BCB11022394667
:10B300006846FDF70FF9360B012368462D0B3946C9
:10B310008DF800300194ADF80860ADF80A50A047F0
:10B320003846D6E70A20D4E70620D2E72046D0E701
:10B33000F4350020702C002018DF704730B585B040
:10B34000054610220C4668460021FDF7EBF8A408DC
:10B35000684601950294FFF7EFFF05B030BD1FB5B9
:10B360009208C2F3090353B90123CDE902026846EA
:10B37000CDE90031FFF7E0FF05B05DF804FB0920DF
:10B38000FAE71FB50023CDE9013303936846022392
:10B390000093FFF7D1FF05B05DF804FB1FB5032351
:10B3A000CDE900309208684602910392FFF7C4FF8E
:10B3B00005B05DF804FB000009B9034B1970034B9D
:10B3C0001B6803B118477047F8350020FC35002092
:10B3D000204B21491A68214B00BF00BF00BF00BFAE
:10B3E00000BF00BF00BF00BF8A422FD000BF00BF18
:10B3F00000BF00BF00BF00BF00BF00BF00BF00BF55
:10B4000000BF00BF00BF00BF00BF00BF00BF00BF44
:10B4100000BF00BF00BF00BF00BF00BF00BF00BF34
:10B4200000BF00BF00BF00BF00BF00BF00BF00BF24
:10B4300000BF00BF00BF00BF00BF00BF00BF00BF14
:10B4400000BF00BF00BF00BF00BF00BF013BC3D1B2
:10B45000704700BF642C00200024F400A086010087
:10B4600008B5FEF7F7FB00B908BDFFF7B1FFFDF720
:10B470002DFEF6E7002258210148FEF715BA00BF5D
:10B4800004360020F8B51B4C06462546237893B9B0
:10B4900001232370184B194C1E60FFF7E1FF0022B7
:10B4A00001212046FFF7FCFE0728F6D040B100231B
:10B4B0002B700320F8BDFFF78BFFFDF707FEE5E7D4
:10B4C000FFF7D8FF0E490F4F08604FF4AE720E48D9
:10B4D0000D4E0A4C01F0BBFFFFF7C2FF3B4657225F
:10B4E00031462046FFF794FE0728F5D00028E1D02A
:10B4F000DDE700BFF8350020FC35002000F0070034
:10B5000000360020B9B307005C37002010B5114B9E
:10B51000114C124900221A7020464FF4AE7201F00D
:10B5200096FF226801320FD14FF4AE7200210A4813
:10B53000FCF7F8FF012300206360FFF7A3FF40B191
:10B54000BDE81040FDF74BBCFFF794FF2368834232
:10B55000EAD110BDF83500200036002000F00700C9
:10B5600070B5084E084CA41BE4080025A54201D183
:10B57000002070BD56F8353098470028F9D10135C4
:10B58000F4E700BF802C0020882C002070B5084E06
:10B59000084CA41BE40800250436A54201D1002074
:10B5A00070BD56F8353098470028F9D10135F4E7D9
:10B5B000802C0020882C0020044A0023C0E900339E
:10B5C0008360C2E90C33C2E90433704700360020BF
:10B5D0002DE9F041184E1949726B336B02F6FF7476
:10B5E000E41A0C40A50805F6FF7503F580570D40D9
:10B5F00003EB00080AB193421BD02A464146384665
:10B60000FFF7ADFE98B92A4641463846FFF7C6FE19
:10B6100068B9A542736B8CBF0446641B1B1B0020DA
:10B620002F44A8443363FFF72DFF002CE5D1BDE87C
:10B63000F0810020FBE700BF0036002000F0FFFF94
:10B6400070B50D4B0D685C6B2D1B04440E462A46ED
:10B6500021460A48FFF7A2FE014638B93046FFF7F7
:10B66000ABFFBDE870400846FFF70CBF29462046F7
:10B67000BDE87040FFF762BE003600200080070082
:10B680002DE9F04743F2080380461E684D4B1A69C6
:10B69000012A994614D05B6993B1D9F8185005F680
:10B6A000FF7525F47F6525F00F05354409F1240762
:10B6B000BB68A52B6ED007D8012B14D0002478E0EE
:10B6C000354609F11807F3E7AA2B75D0AC2BF5D155
:10B6D0002846FFF77DFF0446002867D139462846F3
:10B6E000FFF7AEFF61E0D9F81430012BE6D1D9F8AD
:10B6F0003070D9F824A03E44AAEB0707B7F5805F65
:10B700004FF000024FF001013046B84628BF4FF419
:10B710008058FFF7C5FD044600284AD1034642463B
:10B7200029463046FFF774FD0446002841D14246C1
:10B7300029463046FFF732FE0446D0BB02460121BF
:10B740002846FFF7ADFD044698BBD9F83030434496
:10B75000C9F83030FFF796FEB7EB0807464445447A
:10B76000CCD143F208033A4651461868FEF79CF8DC
:10B77000D9F82830984204BF0123C9E907031248C9
:10B7800008BFC9F818A0FFF717FF0020BDE8F04771
:10B79000FFF778BE2846FFF71BFF044630B938464E
:10B7A000FFF70AFF2046FFF76DFE04460123C8F8A5
:10B7B00000302046BDE8F08739462846BDE8F0470E
:10B7C000FFF73EBF003600202436002010B50B4C9A
:10B7D000236A012B0DD8E3696BB143F20803002201
:10B7E0001868A169FEF760F8E3691B1A58425841CE
:10B7F00010BD0020FCE70120FAE700BF0036002062
:10B8000070B5194C43F2080325681B68A5F540552F
:10B81000ED1A854201D2042070BD1360134B1E6ADD
:10B82000012E1CD19C6904F6FF7424F47F6424F07B
:10B830000F042D1BA84205D90029ECD1C3E90461EE
:10B84000183306E00021C3E9041611680C441460A3
:10B85000243300221860C3E901221046DCE70022ED
:10B86000C3E90422ECE700BF1410001000360020EA
:10B870000023C0E90232C0E900118B781A4402614A
:10B8800091F903301A4442610878003018BF012052
:10B89000704710B542681178034600293AD002F18A
:10B8A0000C014160147B2CB9C2680168FFF7E0FF0E
:10B8B000204610BD5078117900F03004302C1BD197
:10B8C000547B04F03004302C1ED190781969091A89
:10B8D00019610021507810F0300F02BF98680130D4
:10B8E0009860907B084419690144196192F90F200E
:10B8F000114459610120DCE700F0F004202C03D151
:10B90000507910FB01F1E5E700F0C000802808BF86
:10B910000421DFE70846CCE770B5456804460E46CB
:10B9200063681A78B24204D15B7803F00F03082BE6
:10B9300007D12046FFF7ADFF6368AB42F0D100208E
:10B9400070BD0120FCE743681A44426011B101391F
:10B950009A4201D10120704713F8010B01F8010F41
:10B96000F6E770B54268527802F00F01082986B0F8
:10B9700003461FD103691C6800260CB906B070BDD0
:10B98000236826739D68626829466846FFF770FF42
:10B990006368049304F10C0305936B7803F0C00310
:10B9A000802B08BF231D684608BF0493FFF7D9FF0B
:10B9B000A468E2E712F0C00120D102F030001028A4
:10B9C0000ED15A6911705A6818695378946803F057
:10B9D0000F03072B09D10146204600F017F8CDE7E9
:10B9E0009006F0D55B691970C8E71279214614B149
:10B9F00001F02DFDC2E7FCF795FDBFE78029BDD121
:10BA00000069002192060160B8D5EBE77FB50A46D0
:10BA100001466846FFF72CFF30B16846FFF7A1FFEB
:10BA20006846FFF736FFF7E707B05DF804FB10B58F
:10BA3000012203680446984710B1A368013BA36044
:10BA400010BD2DE9F34183680746884623B90026D7
:10BA5000304602B0BDE8F0810DF10701FFF7E7FFC6
:10BA600006460028F3D09DF80740220616D504F0BC
:10BA70007F040725BB68002BE9D00DF1070138468C
:10BA8000FFF7D5FF0028E2D09DF8072002F07F03E2
:10BA9000AB401C43130605F1070502D4C8F800406B
:10BAA000D6E7232DE6D1D2E730B5044685B015465A
:10BAB000A9B90268114B9A4211D0102D06D82A4616
:10BAC00069462046FFF7F0FF05B030BD10226946F9
:10BAD0002046FFF7E9FF0028F6D0103DEDE7A36808
:10BAE000AB4201D20020EFE723682A462046984760
:10BAF0000028F7D0A3685D1BA560E5E747B90700FC
:10BB0000F7B50E4601A907461546FFF79AFFA8B1FB
:10BB1000019A0123D3184FF0000404D2717801F088
:10BB2000C001802901D1204608E031799942FAD339
:10BB300029463846FFF7B8FF019BEC5403B0F0BD2F
:10BB400073B50D4601A906461446FFF77AFF90B17A
:10BB5000019AFF2A11D86B7803F0C003802B02F101
:10BB600001010AD02B798B4207D32146304601F8D8
:10BB7000012BFFF799FF02B070BD0020FBE700002A
:10BB800010B5034C82600022C0E90041C26010BDC4
:10BB900047B907002DE9F347002580460F462E469A
:10BBA0002C46D8F8083023B30DF107014046FFF7C3
:10BBB0003EFFF0B19DF807C00CF07F025FFA82F9FA
:10BBC000A4F12003C4F1200109FA03F329FA01F1D9
:10BBD00009FA04F20B431CF0800F45EA020546EA1D
:10BBE000030604F1070402D1C7E9005602E0462C1F
:10BBF000D7D1002002B0BDE8F08773B50C46694686
:10BC00001646FFF7C7FF68B12379082B0CD1DDE991
:10BC10000045C6E90045DDE90023AB4206BFA2426C
:10BC20000120002002B070BD042B04D1009B3360C2
:10BC30001C460025EFE7022B4FF0000004D1009BCB
:10BC400033809CB20546E6E7012BEBD1009B3370B5
:10BC500003F0FF04F6E737B50D4669461446FFF7D3
:10BC600099FF30B12A79082ADDE9003103D1C4E90E
:10BC7000003103B030BD042A18464FEAE37108D101
:10BC800023601A460B468B4206BF824201200020E9
:10BC9000EFE7022A04D11BB223801AB2D317F2E7CE
:10BCA000012A03D15BB223705AB2F7E70020E0E724
:10BCB000F7B50C46002119702170116001A90746E3
:10BCC00015461E46FFF7BDFE30B9BB6813B9012308
:10BCD0003370002003B0F0BD01990029F7D0CB08E4
:10BCE00001F007012B602170F4E713B50446052924
:10BCF0001FD8DFE801F0030F151E1E1C012201A949
:10BD00002046FFF7D1FE18B19DF90430002BF5DB7A
:10BD100002B010BD082200212046FFF7C5FEF7E75C
:10BD200001A9FFF78EFE0028F2D0019AF3E7042262
:10BD3000F1E70020ECE773B50D4601A90446FFF7D3
:10BD400080FE064618B90026304602B070BD94E861
:10BD50000F0085E80F0001998A42F4D3A960A36817
:10BD60005B1AA360F0E700002DE9F04355686B789B
:10BD700013F0C00489B006468C46174603D0402C09
:10BD80006AD000240AE003F00F025E4903F030039A
:10BD9000102B51F8228020D004D8CBB1204609B016
:10BDA000BDE8F083202B1ED0302BF7D17B6929789A
:10BDB0001970072A0AD17B6838691A792146FCF77D
:10BDC000B1FB7B6839699868FFF720FE3A6940E06B
:10BDD0003A692946C0470446E0E77B6901221A70A8
:10BDE0003A697968F6E7BCF1020FD7F8149024D1CC
:10BDF000042A22D804A9FFF79EFF04460028C0D0D9
:10BE0000069B2BB1796899F800304A799A4205D897
:10BE1000059B7360069B002BC0D0B2E708793A6996
:10BE200000FB032204A8C04728B199F80030013371
:10BE300089F80030E4E70446EAE799F800306A79C7
:10BE40009A429ED93A692979581C89F8000001FB69
:10BE5000032279683046BDE7D2F81080454655F890
:10BE6000043B13B9FFF741FFB5E7022914D104A938
:10BE7000FFF761FF002884D0D8F8003079682A469F
:10BE800004A89847044600283FF47BAF069B002B8C
:10BE9000F2D1059B736081E701292BD04CB24CB1E4
:10BEA00005297FF46EAF04220DEB0201FFF7FCFDC4
:10BEB000042424E00DF1040901340B2C3FF461AF9C
:10BEC000012249463046FFF7EFFD00283FF459AF05
:10BED00019F9013B002BEFDB0B4B049301ABCDE9D0
:10BEE000053400230793D8F8003079682A4604A85F
:10BEF000984770E7082201A9FFF7D6FD082400281B
:10BF0000EAD13EE750D8070047B907002DE9F04FC6
:10BF100091B00446002604A8CDE90266FFF7A8FC0C
:10BF2000A3683BBBDDE9053404A85D78FFF7B1FCED
:10BF30000028F7D115F0300F03D1059B1B7803B112
:10BF40000134002C00F0A9806309002202A9934269
:10BF500040F09C8010AA02EB830304F01F04C4F19C
:10BF600020044FF0FF3053F8383CE040C31A5842E9
:10BF700058410DE00DF1030301AA0DF10201204625
:10BF8000FFF796FE38B99DF80330002BCAD1002088
:10BF900011B0BDE8F08F019904A8FFF7BDFC00289F
:10BFA00050D1019BB3427DD3059D059A537803F090
:10BFB0000F03082B7FD004A8FFF76BFC059B9D4265
:10BFC000F3D14FF0FF36019FB7426BD3089B9DF82A
:10BFD0000290D4F808801D684FF0010AA368002D74
:10BFE0005DD098459CD12B68D3F800B0BBF1000F11
:10BFF00008D04B463A4629462046D8470028C6D0A6
:10C00000AD68EBE7D3F808B09BF800309F42F7D15A
:10C010006A6859460AA8FFF72BFC6B680E9305F176
:10C020000C030F939BF8013003F0C003802B04BF77
:10C030002B1D0E930AAA85F80CA049462046FFF74F
:10C0400093FEDBE7059B5B7813F0300F0FD1069A68
:10C050003F2A0CD8510910AB03EB810102F01F02FB
:10C060000123934051F8382C134341F8383CE568DC
:10C070002DB104AB9DF8022001992046A84704AADF
:10C080009DF802102046FFF76FFE10E051F8225095
:10C0900001357FF47DAF013259E7012078E79845FB
:10C0A0007FF43EAF9DF802102046FFF71EFE0028E9
:10C0B0007FF436AF6BE7167885E770B50C46064619
:10C0C000154611462046FFF7A1FC2A462146304678
:10C0D000BDE87040FFF71ABFF0B585B00C468D681B
:10C0E000694607461646FFF726FE68B1A06858B1B4
:10C0F000637803F03003202B32462946684605D189
:10C10000FFF7DBFF019B7B6005B0F0BDFFF7FEFE94
:10C11000F8E7D3B50C466946FFF73CFD80B1DDE991
:10C12000001300274A0801F0010642EAC37256EAEA
:10C1300007014FEA53031CBFD243DB43C4E900238A
:10C1400002B0D0BD37B50D4669461446FFF7E1FF92
:10C1500068B12B79082B0CD1DDE90001C4E900019D
:10C16000DDE900238B4206BF82420120002003B09C
:10C1700030BD042B03D100982060C117F0E7022BDB
:10C1800004D1BDF90000208000B2F6E7012B04D1F4
:10C190009DF90000207040B2EFE70020E7E713B5FB
:10C1A00004220C460DEB0201FFF77EFC08B1019B57
:10C1B000236002B010BD1146FFF7F1BF13B508228E
:10C1C0000C466946FFF770FC18B1DDE90023C4E9AD
:10C1D000002302B010BD1146FFF7F0BF8B180244D8
:10C1E0008B4200D1704713F8010D02F8010DF7E7FB
:10C1F00010B5013A52B2130601D5002010BD50F817
:10C20000224051F822309C4205D802F1FF32F2D28E
:10C210004FF0FF30F2E70120F0E7000000000000DF
:10C22000C3F10803DB0070B50133002403A500BF90
:10C230005B1920C940CAAD1920C0184720C940CA9F
:10C24000754120C020C940CA754120C020C940CADC
:10C25000754120C020C940CA754120C020C940CACC
:10C26000754120C020C940CA754120C020C940CABC
:10C27000754120C06441204670BD00BF0000000031
:10C28000C3F10803DB0070B50133002403A500BF30
:10C290005B1920C940CAAD1B20C0184720C940CA3D
:10C2A000B54120C020C940CAB54120C020C940CAFC
:10C2B000B54120C020C940CAB54120C020C940CAEC
:10C2C000B54120C020C940CAB54120C020C940CADC
:10C2D000B54120C06441B4FA84F0400970BD00BF8C
:10C2E0002DE9F04F08B4F8CA04B451F8042BA3FBAD
:10C2F000028940F8048B4FF0000AE4FB629A4FF089
:10C30000000BE5FB62AB4FF0000CE6FB62BC4FF0AC
:10C31000000EE7FB62CE51F8042B4FF00008E3FB60
:10C32000628940F8048BE4FB629AE5FB62ABE6FBB2
:10C3300062BCE7FB62CE51F8042B4FF00008E3FB30
:10C34000628940F8048BE4FB629AE5FB62ABE6FB92
:10C3500062BCE7FB62CE51F8042B4FF00008E3FB10
:10C36000628940F8048BE4FB629AE5FB62ABE6FB72
:10C3700062BCE7FB62CE51F8042B4FF00008E3FBF0
:10C38000628940F8048BE4FB629AE5FB62ABE6FB52
:10C3900062BCE7FB62CE40F8049B40F804AB40F877
:10C3A00004BB40F804CB40F804EB0CBC052B00F0B8
:10C3B0001E810C68A0F11400A1F11401A2F1140275
:10C3C00052F804EB4FF0000550F8046BE4FB6E5696
:10C3D00052F804EB50F8047BE4FB6E6752F804EB70
:10C3E00050F8048BE4FB6E7852F804EB50F8049B91
:10C3F000E4FB6E8952F804EB50F804ABE4FB6E9A50
:10C40000A0F1140052F8044B51F804EB4FF0000C6B
:10C41000E4FB6EC540F804CB51F804EBE4FB6E5628
:10C4200040F8045B51F804EBE4FB6E6740F8046BE2
:10C4300051F804EBE4FB6E7840F8047B51F804EB10
:10C44000E4FB6E8940F8048B51F804EBE4FB6E9A30
:10C45000A0E80006062B00F0CA800C68A0F11800C6
:10C46000A1F11801A2F1180252F804EB4FF00005F7
:10C4700050F8046BE4FB6E5652F804EB50F8047B62
:10C48000E4FB6E6752F804EB50F8048BE4FB6E7823
:10C4900052F804EB50F8049BE4FB6E8952F804EB6D
:10C4A00050F804ABE4FB6E9A52F804EB50F804BB6E
:10C4B000E4FB6EABA0F1180052F8044B51F804EB0A
:10C4C0004FF0000CE4FB6EC540F804CB51F804EBD0
:10C4D000E4FB6E5640F8045B51F804EBE4FB6E6736
:10C4E00040F8046B51F804EBE4FB6E7840F8047BF1
:10C4F00051F804EBE4FB6E8940F8048B51F804EB2F
:10C50000E4FB6E9A40F8049B51F804EBE4FB6EAB3D
:10C51000A0E8000C072B6AD008B40C68A0F11C003E
:10C52000A1F11C01A2F11C0252F804EB4FF000052E
:10C5300050F8046BE4FB6E5652F804EB50F8047BA1
:10C54000E4FB6E6752F804EB50F8048BE4FB6E7862
:10C5500052F804EB50F8049BE4FB6E8952F804EBAC
:10C5600050F804ABE4FB6E9A52F804EB50F804BBAD
:10C57000E4FB6EAB52F804EB50F804CBE4FB6EBC6A
:10C58000A0F11C0052F8044B51F804EB4FF00003EB
:10C59000E4FB6E3540F8043B51F804EBE4FB6E56C7
:10C5A00040F8045B51F804EBE4FB6E6740F8046B61
:10C5B00051F804EBE4FB6E7840F8047B51F804EB8F
:10C5C000E4FB6E8940F8048B51F804EBE4FB6E9AAF
:10C5D00040F8049B51F804EBE4FB6EAB40F804AB6D
:10C5E00051F804EBE4FB6EBCA0E8001808BCBDE801
:10C5F000F08F2DE9F04FB1E8005E06B4AAFB0912F6
:10C600004FF00003EBFB69234FF00004ECFB6934AF
:10C610004FF00005EEFB69454FF00006EBFB6A6347
:10C62000ECFB6A344918524176415B41A9FB097819
:10C630004FF0000949F1000918EB0108A0E880015A
:10C64000AAFB0A78574158EB0608A0E88001EEFBE8
:10C650006A454FF0000A4AF1000A4FF00001ECFB76
:10C660006B14EEFB6B454FF00002EEFB6C255FEAAE
:10C6700059094941644152416D4149F10009EBFBBF
:10C680006B3A1AEB010AA0E80804ACFB0C6A66419D
:10C690005AEB020AA0E84004AEFB0E6A6E415AEB68
:10C6A000090AA0E8400406BC052A00F0E680A0F1D3
:10C6B0001400A1F11401B1E8E043A5FB0E344FF0E2
:10C6C0000005E6FB6E454FF00006E7FB6E564FF0A7
:10C6D0000007E8FB6E674FF00008E9FB6E784FF04B
:10C6E0000009DB1864416D4176417F4158EB080831
:10C6F00059F1000950F804CB13EB0C0350F804CBAC
:10C7000054EB0C0450F804CB55EB0C0550F804CB5B
:10C7100056EB0C0650F804CB57EB0C0758F1000809
:10C7200059F10009A0F11400EEFB0E89A0E8F8030E
:10C73000062A00F0A280A0F11800A1F11801B1E8CA
:10C74000E047A5FB0E344FF00005E6FB6E454FF0C9
:10C750000006E7FB6E564FF00007E8FB6E674FF0F0
:10C760000008E9FB6E784FF00009EAFB6E894FF094
:10C77000000ADB1864416D4176417F4158EB08089F
:10C7800059EB09095AF1000A50F804CB13EB0C03DA
:10C7900050F804CB54EB0C0450F804CB55EB0C05CB
:10C7A00050F804CB56EB0C0650F804CB57EB0C07B3
:10C7B00050F804CB58EB0C0859F100095AF1000A63
:10C7C000A0F11800EEFB0E9AA0E8F807072A54D053
:10C7D000A0F11C00A1F11C01B1E8E04FA5FB0E3453
:10C7E0004FF00005E6FB6E454FF00006E7FB6E5686
:10C7F0004FF00007E8FB6E674FF00008E9FB6E782A
:10C800004FF00009EAFB6E894FF0000AEBFB6E9ACD
:10C810004FF0000BDB1864416D4176417F4158EBCE
:10C82000080859EB09095AEB0A0A5BF1000B50F8AA
:10C8300004CB13EB0C0350F804CB54EB0C0450F86E
:10C8400004CB55EB0C0550F804CB56EB0C0650F816
:10C8500004CB57EB0C0750F804CB58EB0C0850F8FE
:10C8600004CB59EB0C095AF1000A5BF1000BA0F163
:10C870001C00EEFB0EABA0E8F80FBDE8F08F002324
:10C8800010B51C465AB2914200DC10BD40F823405E
:10C890000133F7E72DE9F0471F46B3F90230894627
:10C8A00013F11F0148BF03F13E014D11D91D48BFCF
:10C8B00003F10E01CC1094424FFA85F828BF1446BC
:10C8C00041460646FFF7DBFF22464946FFF786FC56
:10C8D000B7F90220E40094421FD9A41A06EB85019F
:10C8E0000022C4F120058E420ED324374246314641
:10C8F0003846FFF77DFC01280FD043463A463046C4
:10C90000BDE8F047FFF7BCBC51F8040D20FA04F372
:10C9100013430B6000FA05F2E5E7BDE8F08710B5B8
:10C9200000231A465CB2A14203DCB2FA82F040094D
:10C9300010BD50F8234001332243F3E74A1101238D
:10C9400050F8220001F01F0103FA01F1084070477E
:10C95000013910B549B2041D0A06CBB204D401391D
:10C9600054F82120002AF7D001335BB273B103F1F0
:10C970008042013A50F82220002022B9013B00EB0E
:10C98000431318B210BD52080130F6E71846F9E714
:10C9900010B500235CB2A24200DC10BD51F8234068
:10C9A00040F823400133F5E7F0B5082289B00C4682
:10C9B0000646FFF7EDFFCB6A03930B6B04934B6BBB
:10C9C00005938B6B0693CB6B0793002708236A466E
:10C9D00069466846CDE901770097FFF721FC0823F7
:10C9E00005466A4631463046FFF71AFC236B03932F
:10C9F000636B0493A36B0593E36B0544CDE90637A2
:10CA00006A46082369466846FFF70AFC082305447E
:10CA10006A4631463046FFF703FC236A0093636A97
:10CA20000193A36A0293A36B0693E36B07930544F8
:10CA300008236A4631463046CDE904770397FFF76D
:10CA4000EFFB636A0093A36AA26B0193E36A02930C
:10CA50000492636BE26B0393CDE90523236A07938A
:10CA6000054408236A4631463046FFF7D9FBE36A9E
:10CA70000093236B0193636B0293236A0693A36A6B
:10CA80000793054408236A4631463046CDE90477CA
:10CA90000397FFF7F5FB236B0093636B0193A36B85
:10CAA0000293E36B0393636A0693E36A07932D1A79
:10CAB00008236A4631463046CDE90477FFF7E0FBAC
:10CAC000636B0093A36B0193E36B0293236A03935D
:10CAD000636A0493A36ACDE90537236B07932D1A84
:10CAE00008236A4631463046FFF7CAFBA36B009322
:10CAF000E36BCDE90137636A0393A36A0493E36AA6
:10CB0000CDE90537636B07932D1A08236A46314632
:10CB10003046FFF7B5FB2D1A0D4C0FD435B908225E
:10CB200031462046FFF764FB01280FD00823224638
:10CB300031463046FFF7A4FB2D1AEFE708232246C3
:10CB400031463046FFF76CFB2D18F7D409B0F0BD25
:10CB500078D8070030B5013A52B20023140603D545
:10CB6000B3FA83F0400930BD50F8224051F822500A
:10CB70006C402343013AF1E700EB81010023884236
:10CB800000D3704751F8042D43EA52030B60D307DA
:10CB9000F5E770B5036813F001050646144605D0A5
:10CBA00013460A460146FFF73BFB05462146304641
:10CBB000FFF7E2FF45B104F18042013A56F8223016
:10CBC00043F0004346F8223070BD70B59DF9104027
:10CBD0001E4623460546FFF723FB30B92246294669
:10CBE0003046FFF705FB012807D023463246294689
:10CBF0002846BDE87040FFF743BB70BD70B59DF996
:10CC000010401E4623460546FFF73AFB38B123463F
:10CC1000324629462846BDE87040FFF701BB70BD8B
:10CC20002DE9F04FA5B01D4614ABCDE90231814688
:10CC3000294610461746FFF78BFEC0EB851004B25D
:10CC4000002C2646B8BF04F11F06634246F3471680
:10CC500003F01F0304F01F0804A858BFC3F1000825
:10CC60003146FFF70CFEB8F1000F30B22DDD04ABFA
:10CC7000002203EB8000C8F1200C13469D4219D816
:10CC80002FB27B00019304AB03EB870705F1FF385C
:10CC900024AB012603EB8808002C54DA24AB03EB09
:10CCA00086062A4656F8881C4846FFF771FE25B0CE
:10CCB000BDE8F08F57F8236006FA08F10A4340F800
:10CCC000042B013326FA0CF2D8E704AB2A46394686
:10CCD00003EB8000FFF75CFED2E70FFA82FE5AF802
:10CCE000883C53F82EB024AB03EB8202013052F89B
:10CCF000803C0B44BBEB030334BF012200229B4565
:10CD000018BF11465CF8882C42F82E30019B42B2C5
:10CD10009A42E2DB731A5E42294604A85E41FFF79D
:10CD20002BFF24AB03EB8503294653F8802C58F8DE
:10CD3000803C384643EAC273013C48F8803C24B248
:10CD4000FFF71AFFA8E724AB0020C6F1010C01464B
:10CD500003EB860A03EB8C0CD8E770B590B0054660
:10CD60009DF950401E4668462346FFF7B9FA324601
:10CD700069462846FFF754FF10B070BD30B51C4619
:10CD800091B0054693F900306846FFF7A9FAD4F848
:10CD9000AC3069462846984711B030BD30B51446CE
:10CDA00091B0054692F900206846FFF722FCD4F8BE
:10CDB000AC3069462846984711B030BD2DE9F041A6
:10CDC00015468AB0044688461C22002103A8FBF7BA
:10CDD000A9FB2E1D95F9007003232A4641462046E3
:10CDE0000293FFF7DBFF334602AA21462046009755
:10CDF000FFF704FF2B46424621462046FFF7BEFFC1
:10CE00000097334605F1840221462046FFF7DDFEF8
:10CE10000AB0BDE8F0812DE9F04793F9006092B0C7
:10CE2000044689461046314615469846FFF777FD79
:10CE3000002840F091804246494602A8FFF7AEFF25
:10CE4000434602AA21460AA8FFF798FF02A908460E
:10CE50004246FFF7A3FF43462A4649464846FFF7A6
:10CE60008DFF08F10407424629462846FFF796FF42
:10CE70003B462A46214620460096FFF7A6FE3B4643
:10CE80002A46294628460096FFF79FFE3B462A463B
:10CE9000214628460096FFF7B1FE43462A46214622
:10CEA0002046FFF76BFF3B46224621462846009668
:10CEB000FFF78BFE3B4600962A4621462046FFF7A9
:10CEC00084FE2368DB074AD533463A46214620468E
:10CED000FFF7A6F9314682462046FFF74DFE06F1E0
:10CEE0008043013B54F8230040EACA7044F8230011
:10CEF000424621462846FFF751FF3B460AAA2946EB
:10CF000028460096FFF77AFE3B460AAA294628469D
:10CF10000096FFF773FE0AA908463B462A4600968C
:10CF2000FFF76CFE43460AAA21462046FFF726FF7C
:10CF300002AA3B46104621460096FFF75FFE3246A6
:10CF400029462046FFF724FD49462846FFF720FDE5
:10CF500002A94846FFF71CFD12B0BDE8F087314634
:10CF60002046FFF709FEC3E72DE9F0438BB01446D6
:10CF7000129D15F9046B00961F46804689462B4684
:10CF80000246214602A8FFF739FE02A9129A084676
:10CF9000FFF704FF129B02AA41464046FFF7EEFE50
:10CFA000129B02AA21462046FFF7E8FE2B464A467E
:10CFB000394638460096FFF721FE129A394602A8F4
:10CFC000FFF7ECFE02A92B46424608460096FFF703
:10CFD00015FE02A92B46224608460096FFF70EFED4
:10CFE0002B464246214620460096FFF707FE129B3D
:10CFF000224649464846FFF7C1FE2B4602AA414653
:10D0000020460096FFF7FAFD129B22463946384625
:10D01000FFF7B4FE2B464A46394638460096FFF7DE
:10D02000EDFD324602A92046FFF7B2FC0BB0BDE889
:10D03000F083F0B5154689B01C4607460E461A46E1
:10D0400029466846FFF7AAFE23466A46394638460F
:10D05000FFF794FE23462A4669466846FFF78EFE90
:10D0600023466A4631463046FFF788FE09B0F0BDD8
:10D07000F0B50F46A1B006461946384615461C467F
:10D08000FFF74DFC20B13046FFF7F9FB21B0F0BDB2
:10D09000224639466846FFF77BFC294608A8FFF779
:10D0A00077FC10A82146FFF7EAFB012318A810938C
:10D0B000FFF7E5FB224608A96846FFF799F828B96B
:10D0C000224610A93046FFF763FCDFE7009BDA0732
:10D0D00009D421466846FFF74FFD2246294610A88D
:10D0E000FFF757FDE6E7089BDB0707D4214608A8B2
:10D0F000FFF742FD2246294618A8F1E700282346FB
:10D100001CDD08AA69466846FFF7BAF8214668465A
:10D11000FFF732FD224618A910A8FFF769F800288A
:10D1200005DA10A923462A460846FFF779F810A920
:10D13000234618AA0846FFF7A3F8CEE708A96A46CF
:10D140000846FFF79DF8214608A8FFF715FD22467F
:10D1500010A918A8FFF74CF8002805DA18A92346EB
:10D160002A460846FFF75CF818A9234610AA084685
:10D17000FFF786F8BEE700000048704774D8070044
:10D180002DE9F04FEDB01F46769E0490B6F90230BF
:10D1900096F9005013F11F0948BF03F13E0949F306
:10D1A000471909F1FF3824AB002443F828406CAB41
:10D1B00003EB88034CA88A469346394696F901202A
:10D1C00043F8804C43F8604CFFF708F896F90120CB
:10D1D00054A8B918FFF702F829464CA8FFF79FFB9F
:10D1E0000746002840F01F8154A8FFF798FB0390E2
:10D1F000002840F01A8106F124034A464CA918463B
:10D200000293FEF7F5FF012840F011814A4654A928
:10D210000298FEF7EDFF0128069040F008811CAC53
:10D220000CAF4B46029A54A92046FFF721FF039BFF
:10D2300047F828305A46514638463346FFF72AFB0E
:10D2400039463846029BCDF800902246FFF785FD0F
:10D250000DF5B878029BCDF8009022464CA914A891
:10D26000FFF77BFD2A4640460499FFF791FBAB0090
:10D2700008EB030A0793049BA900591806F1440B15
:10D280005046FFF785FB594634A8FFF781FBAB00FA
:10D290000BEB03013CA8FFF77BFB331D414634AA8F
:10D2A000204600950593FFF7A9FC534642463CA94A
:10D2B00034A80096FFF758FE2B46321D2146204623
:10D2C000FFF7D6FE2246514640463346FFF7B1FEF1
:10D2D000039BCDE9083B049B49463846CDE90A3813
:10D2E000FFF736FB4946804614A8FFF731FB80451F
:10D2F000B8BF80461FFA88F808F1FF3B0FFA8BFB96
:10D3000059463846FFF71AFB5946071C14A818BFA0
:10D310000127FFF713FB002814BF022300231F433C
:10D320000DF1200A2A465AF8277024A83946FFF73B
:10D330002FFB0DF1B00BAB00F9185846FFF728FB97
:10D3400029462046FFF79BFAA8F10208069B2360B6
:10D350000FFA88F80DF1900AB8F1000F1FDA2B468A
:10D36000059A21462046FFF783FE3346224659465A
:10D370005046FFF75EFE4A4651460298FEF738FFD8
:10D38000012804D04B46029A5046FEF779FF2A4600
:10D390004CA95046FFF7DEFB6DB0BDE8F08F334679
:10D3A0002246D6F8A47059465046B84741460CA8C4
:10D3B000FFF7C4FA4146071C14A818BF0127FFF75E
:10D3C000BDFA002814BF022300231F4308AB53F803
:10D3D00027701FB32A46394634A8FFF7D9FA079BAE
:10D3E0003CA8F918FFF7D4FA334622463CA934A8E2
:10D3F000FFF71FFE059B009534AA514644A8FFF78E
:10D40000FDFB5B4652463CA934A80096FFF7ACFDF5
:10D41000334644AA21462046FFF7B0FC08F1FF3806
:10D420000FFA88F898E72046B6E73846B4E703983D
:10D43000B2E730B501390024A24201D1002005E055
:10D44000035D01340D5DAB42F6D0581B30BD0A447C
:10D45000914200F1FF3300D1704710B511F8014B34
:10D4600003F8014F9142F9D110BD0000F8B500BF9B
:10D47000F8BC08BC9E467047F8B500BFF8BC08BCB5
:10D480009E467047002C0020011101FF01000000A2
:10D4900000000000021702FE64000000DCD4070058
:10D4A000031704FC040000007CD507000000000006
:10D4B0000000000000000000010100000100000069
:10D4C0000000000002050000210000000000000034
:10D4D000000000000000000000000000011104FC3A
:10D4E0000400000000000000021104FC0400000021
:10D4F00000000000032104FC040400000000000000
:10D50000041101FF0100000000000000051102FEEF
:10D510000400000000000000061104FC04000000EC
:10D5200000000000071104FC0400000000000000DF
:10D53000081701FF22000000B8D40700091001FFFE
:10D540000100000054D507000000000000000000AA
:10D550000000000000000000011704FC7000000043
:10D5600088D40700021704FCB400000094D507001B
:10D5700000000000000000000000000001010000A9
:10D580000400000000000000000000000000000097
:10D5900000000000010700007000000088D40700B0
:10D5A000020100000100000000000000030500006F
:10D5B000410000000000000000000000000000002A
:10D5C000000000004901B952C5EF41DE27476A5506
:10D5D00027B31CE72D1ECB0FA00C3792BE6AB2E911
:10D5E0009B2403956593690B5EF09CFDA5C02CEE12
:10D5F000F1ECA5A1470A9B3F814C5FD407D8A31447
:10D6000004C609D3C4D50700400000005245414478
:10D610005920544F205550444154450D0A00444967
:10D6200053434F4E4E45435445440D0A00424F4F1D
:10D63000544C4F414445520D0A0052454C4541530C
:10D64000452042544E3120464F52204446550D0A43
:10D65000003C2020202020202020202020202020CE
:10D66000202020202020203E0D003D000D0A4446B1
:10D670005520535441525445440D0A000400000003
:10D680000004010000000402000000040300000088
:10D69000040400000004050000000406000000046B
:10D6A0000700000004080000000409000000040A4C
:10D6B000000000040B000000140C000000040D002A
:10D6C0000000040E000000040F0000000410000021
:10D6D0000004110000000412000000041300000008
:10D6E00004140000000415000000041600000004EB
:10D6F0001700000004180000000419000000041ABC
:10D70000000000041B000000041C240013041D0082
:10D710000003041E000000041F000000982F8A422E
:10D7200091443771CFFBC0B5A5DBB5E95BC2563973
:10D73000F111F159A4823F92D55E1CAB98AA07D88B
:10D74000015B8312BE853124C37D0C55745DBE72AE
:10D75000FEB1DE80A706DC9B74F19BC1C1699BE42E
:10D760008647BEEFC69DC10FCCA10C246F2CE92DBE
:10D77000AA84744ADCA9B05CDA88F97652513E98E2
:10D780006DC631A8C82703B0C77F59BFF30BE0C6E9
:10D790004791A7D55163CA0667292914850AB72777
:10D7A00038211B2EFC6D2C4D130D385354730A6514
:10D7B000BB0A6A762EC9C281852C7292A1E8BFA2EB
:10D7C0004B661AA8708B4BC2A3516CC719E892D153
:10D7D000240699D685350EF470A06A1016C1A419D6
:10D7E000086C371E4C774827B5BCB034B30C1C39D5
:10D7F0004AAAD84E4FCA9C5BF36F2E68EE828F7494
:10D800006F63A5781478C8840802C78CFAFFBE90AD
:10D81000EB6C50A4F7A3F9BEF27871C63C3300203C
:10D82000193300202000000001000000000000006B
:10D8300050EADA308883B89F604F15F30000C98E34
:10D84000001002004466755461726700E4330020E2
:10D8500057BC0700FBBB070045C10700B7C1070065
:10D86000D7C1070041BB070001BB0700D9C00700B3
:10D870000000000008200001FFFFFFFFFFFFFFFF87
:10D88000FFFFFFFF0000000000000000000000009C
:10D8900001000000FFFFFFFF512563FCC2CAB9F37E
:10D8A000849E17A7ADFAE6BCFFFFFFFFFFFFFFFF57
:10D8B00000000000FFFFFFFF96C298D84539A1F491
:10D8C000A033EB2D817D0377F240A463E5E6BCF83D
:10D8D00047422CE1F2D1176BF551BF376840B6CB08
:10D8E000CE5E316B5733CE2B169E0F7C4AEBE78E04
:10D8F0009B7F1AFEE242E34F4B60D2273E3CCE3B79
:10D90000F6B053CCB0061D65BC86987655BDEBB31A
:10D91000E7933AAAD835C65A17CE0700BDCD0700FF
:08D92000A9C907000000000086
:08D9280018ABFF7F01000000B5
:10D9300000000000000000000000000000000000E7
:10D9400000000000000000000000000000000000D7
:10D9500000000000000000000000000000000000C7
:10D9600000000000000000000000000000000000B7
:10D9700000000000000000000000000000000000A7
:10D980000000000000000000000000000000000097
:10D990000100FFFF0090D0032584070001840700E9
:10D9A0000010000000300800BDB1070000000000BA
:08D9B000B1A8070055A2070011
:020000020000FC
:020000041000EA
:041014000080070051
:0410180000E00700ED
:0400000370008539CB
:00000001FF
